:020000040000FA
:10000000006AD2EF00F0E950086E819680988098DF
:10001000939692989298F00E9216085000B220D0C3
:100020003A0E026EFC0EA0EC00F0330E076E2ED8D6
:10003000100E026E680EA0EC00F028D8640E9FEC43
:1000400000F0220E076E22D8280E09D80C0E07D811
:10005000010E05D8060E03D80082085001D000809A
:10006000076E00A00BD0809803080EE30DD8070E92
:10007000026ED00EA0EC00F0D88012000080FE08C6
:10008000D8B4CFEF00F08088073A00A000908186B6
:10009000F00E801607500F0B80128196073A00B0C1
:1000A000F5D7320E9FEC00F0D8801200139E0A5054
:1000B000D8B4138E100E096EE86A05360636E83499
:1000C00021D80966F9D71200139E0A50D8B4138EAE
:1000D000050E096E270E046E100E0CD8030E046E6A
:1000E000E80E08D8046A640E05D8046A0A0E02D81D
:1000F000055008D0036E0650026E0550016EB1EC3B
:1001000000F00150016E094E139E0A5003E0095C95
:10011000D8B012000150D8A4139E13BE1200300FA5
:10012000C9EF00F0046A036EE86A0306045AD8A017
:10013000CFEF00F0030E026EE40E02D8F5D7026A8C
:10014000F50F016EFE0E04E300D004000126FDE26F
:10015000000001260206F9E201A002D000D0000052
:100160001200066A056A100E076E0234053606365E
:100170000350055E0450065A05E20350052604505C
:100180000622D89001360236072EEFD70150CFEF66
:1001900000F0E96EFB6A1250FA6E1150F96E000120
:1001A00004001200956A946A070EC16EC68AC6885A
:1001B000C79C9E96C79E550E1C6E966A010E046ED5
:1001C000F40EB1DFFE0E20DF010E1EDF0A6A1CC036
:1001D00005F0066A060E116E126A68DFFE0E14DF65
:1001E000C00E12DF0A6A1CC005F0066A060E116E08
:1001F000126A6ADF010E046EF40E95DF01EC01F065
:10020000FDD78390C96A9E9604009EB609EF01F05F
:10021000FBD7C9CF1AF0C96A9E9604009EB612EFAA
:1002200001F0FBD7C9CF1BF083801BC084FF010EF8
:0C023000046EF40E78DF12000300FED70D
:020000040030CA
:04000000FF321FF3B9
:020006008BFF6E
:00000001FF
